:020000040000FA
:040000008B01082840
:100010008501073099008316910100308100273057
:10002000850095000F30870000308C00831224304B
:1000300096001930930080309700051205160E21A6
:1000400005120E2105160E2105120E21051C392060
:10005000851C4820051D5720851EF220071C6620A0
:10006000871C8220071D9E20871DBA20871ED62050
:100070002628051600301B2100301B2100301B21D3
:1000800000301B2108301B210E210E210512080013
:10009000051600301B2100301B2100301B210030D1
:1000A0001B2188301B210E210E2105120800051688
:1000B00000301B2100301B2100301B2100301B2190
:1000C00081301B210E210E21051208000516143067
:1000D0001B2143301B2100301B2100301B2101302C
:1000E0001B210E2105120E21051601301B210030A7
:1000F0001B2100301B2100301B2107301B210E214A
:1001000005120800051614301B2143301B21203036
:100110001B2100301B2101301B210E2105120E2155
:10012000051601301B2100301B2100301B2100303F
:100130001B2107301B210E21051208000516143063
:100140001B2154301B2125301B2100301B21013085
:100150001B210E2105120E21051608301B2100302F
:100160001B2100301B2100301B2107301B210E21D9
:1001700005120800051600301B2135301B21803088
:100180001B2100301B2101301B210E2105120E21E5
:10019000051601301B2100301B2100301B210030CF
:1001A0001B2107301B210E210512080005161430F3
:1001B0001B2161301B2100301B2100301B2101302D
:1001C0001B210E2105120E21051601301B210030C6
:1001D0001B2100301B2100301B2107301B210E2169
:1001E00005120800051614301B2162301B21503007
:1001F0001B2100301B2101301B210E2105120E2175
:10020000051601301B2100301B2100301B2100305E
:100210001B2107301B210E21051208006430A200AB
:100220001421A20B10290800FA30A10000000000E0
:0E023000A10B162908008C1C1B299500080044
:02400E00E43399
:00000001FF
